 IndyRedefineClass

 Timestamp is 2ab0b2c4 (reproducible build file hash)

 Preferred load address is 0000000180000000

 Start         Length     Name                   Class
 0001:00000000 00003ac0H .text$mn                CODE
 0001:00003ac0 00000036H .text$mn$00             CODE
 0001:00003af6 00000092H .text$x                 CODE
 0002:00000000 000001f8H .idata$5                DATA
 0002:000001f8 00000038H .00cfg                  DATA
 0002:00000230 00000008H .CRT$XCA                DATA
 0002:00000238 00000008H .CRT$XCZ                DATA
 0002:00000240 00000008H .CRT$XIA                DATA
 0002:00000248 00000008H .CRT$XIC                DATA
 0002:00000250 00000008H .CRT$XIZ                DATA
 0002:00000258 00000008H .CRT$XLA                DATA
 0002:00000260 00000008H .CRT$XLZ                DATA
 0002:00000268 00000008H .CRT$XPA                DATA
 0002:00000270 00000008H .CRT$XPZ                DATA
 0002:00000278 00000008H .CRT$XTA                DATA
 0002:00000280 00000010H .CRT$XTZ                DATA
 0002:00000288 00000000H .gehcont$y              DATA
 0002:00000288 00000000H .gfids$y                DATA
 0002:00000290 00001e70H .rdata                  DATA
 0002:00002100 00000000H .rdata$CastGuardVftablesA DATA
 0002:00002100 00000000H .rdata$CastGuardVftablesC DATA
 0002:00002100 00000028H .rdata$T                DATA
 0002:00002128 000000b0H .rdata$voltmd           DATA
 0002:000021d8 00000320H .rdata$zzzdbg           DATA
 0002:000024f8 00000008H .rtc$IAA                DATA
 0002:00002500 00000008H .rtc$IZZ                DATA
 0002:00002508 00000008H .rtc$TAA                DATA
 0002:00002510 00000008H .rtc$TZZ                DATA
 0002:00002518 00000004H .tls                    DATA
 0002:0000251c 00000004H .tls$                   DATA
 0002:00002520 00000008H .tls$ZZZ                DATA
 0002:00002528 000003b8H .xdata                  DATA
 0002:000028e0 00000350H .edata                  DATA
 0002:00002c30 0000008cH .idata$2                DATA
 0002:00002cbc 00000014H .idata$3                DATA
 0002:00002cd0 000001f8H .idata$4                DATA
 0002:00002ec8 000004baH .idata$6                DATA
 0003:00000000 00000060H .data                   DATA
 0003:00000060 00000978H .bss                    DATA
 0004:00000000 00000408H .pdata                  DATA

  Address         Publics by Value              Rva+Base               Lib:Object

 0000:00000000       __AbsoluteZero             0000000000000000     <absolute>
 0000:00000000       ___safe_se_handler_count   0000000000000000     <absolute>
 0000:00000000       ___safe_se_handler_table   0000000000000000     <absolute>
 0000:00000000       __arm64x_extra_rfe_table   0000000000000000     <absolute>
 0000:00000000       __arm64x_extra_rfe_table_size 0000000000000000     <absolute>
 0000:00000000       __arm64x_native_entrypoint 0000000000000000     <absolute>
 0000:00000000       __arm64x_redirection_metadata 0000000000000000     <absolute>
 0000:00000000       __arm64x_redirection_metadata_count 0000000000000000     <absolute>
 0000:00000000       __dynamic_value_reloc_table 0000000000000000     <absolute>
 0000:00000000       __enclave_config           0000000000000000     <absolute>
 0000:00000000       __guard_check_icall_a64n_fptr 0000000000000000     <absolute>
 0000:00000000       __guard_eh_cont_count      0000000000000000     <absolute>
 0000:00000000       __guard_eh_cont_table      0000000000000000     <absolute>
 0000:00000000       __guard_fids_count         0000000000000000     <absolute>
 0000:00000000       __guard_fids_table         0000000000000000     <absolute>
 0000:00000000       __guard_iat_count          0000000000000000     <absolute>
 0000:00000000       __guard_iat_table          0000000000000000     <absolute>
 0000:00000000       __guard_longjmp_count      0000000000000000     <absolute>
 0000:00000000       __guard_longjmp_table      0000000000000000     <absolute>
 0000:00000000       __hybrid_auxiliary_iat     0000000000000000     <absolute>
 0000:00000000       __hybrid_auxiliary_iat_copy 0000000000000000     <absolute>
 0000:00000000       __hybrid_code_map          0000000000000000     <absolute>
 0000:00000000       __hybrid_code_map_count    0000000000000000     <absolute>
 0000:00000000       __x64_code_ranges_to_entry_points 0000000000000000     <absolute>
 0000:00000000       __x64_code_ranges_to_entry_points_count 0000000000000000     <absolute>
 0000:00000100       __guard_flags              0000000000000100     <absolute>
 0000:00000000       __ImageBase                0000000180000000     <linker-defined>
 0001:00000000       ??1JvmtiResource@@QEAA@XZ  0000000180001000 f i libIndyRedefineClass.obj
 0001:0000008c       ?NewObject@JNIEnv_@@QEAAPEAV_jobject@@PEAV_jclass@@PEAU_jmethodID@@ZZ 000000018000108c f i libIndyRedefineClass.obj
 0001:000000b4       ?SetEventNotificationMode@_jvmtiEnv@@QEAA?AW4jvmtiError@@W4jvmtiEventMode@@W4jvmtiEvent@@PEAV_jobject@@ZZ 00000001800010b4 f i libIndyRedefineClass.obj
 0001:000000c0       ?TranslateError@@YAPEBDW4jvmtiError@@@Z 00000001800010c0 f   libIndyRedefineClass.obj
 0001:00000378       ?nsk_jni_check_exception@@YAHPEAUJNIEnv_@@QEBDH@Z 0000000180001378 f   libIndyRedefineClass.obj
 0001:000004bc       ?nsk_jni_lverify@@YAHHPEAUJNIEnv_@@HQEBDH1ZZ 00000001800014bc f   libIndyRedefineClass.obj
 0001:0000055c       Agent_Initialize           000000018000155c f   libIndyRedefineClass.obj
 0001:00000868       Agent_OnAttach             0000000180001868 f   libIndyRedefineClass.obj
 0001:00000868       Agent_OnLoad               0000000180001868 f   libIndyRedefineClass.obj
 0001:00000870       Java_nsk_share_jvmti_ArgumentHandler_getAgentOptionsString 0000000180001870 f   libIndyRedefineClass.obj
 0001:00000920       Java_nsk_share_jvmti_DebugeeClass_checkStatus 0000000180001920 f   libIndyRedefineClass.obj
 0001:000009a8       Java_nsk_share_jvmti_DebugeeClass_resetAgentData 00000001800019a8 f   libIndyRedefineClass.obj
 0001:00000a08       Java_nsk_share_jvmti_RedefineAgent_agentStatus 0000000180001a08 f   libIndyRedefineClass.obj
 0001:00000a14       Java_nsk_share_jvmti_RedefineAgent_isRedefined 0000000180001a14 f   libIndyRedefineClass.obj
 0001:00000a20       Java_nsk_share_jvmti_RedefineAgent_redefineAttempted 0000000180001a20 f   libIndyRedefineClass.obj
 0001:00000a2c       Java_vm_mlvm_indy_func_jvmti_share_IndyRedefineClass_checkStatus 0000000180001a2c f   libIndyRedefineClass.obj
 0001:00000ad8       Java_vm_mlvm_indy_func_jvmti_share_IndyRedefineClass_setPopFrameDepthAfterRedefine 0000000180001ad8 f   libIndyRedefineClass.obj
 0001:00000ae0       Java_vm_mlvm_indy_func_jvmti_share_IndyRedefineClass_setRedefineTriggerMethodName 0000000180001ae0 f   libIndyRedefineClass.obj
 0001:00000b18       Java_vm_mlvm_indy_func_jvmti_share_IndyRedefineClass_setRedefinedClassFileName 0000000180001b18 f   libIndyRedefineClass.obj
 0001:00000b58       MA_checkStatus             0000000180001b58 f   libIndyRedefineClass.obj
 0001:00000e68       __local_stdio_printf_options 0000000180001e68 f i libIndyRedefineClass.obj
 0001:00000e70       _snprintf                  0000000180001e70 f i libIndyRedefineClass.obj
 0001:000011f8       copyFromJString            00000001800021f8 f   libIndyRedefineClass.obj
 0001:000012e0       exitOnError                00000001800022e0 f   libIndyRedefineClass.obj
 0001:00001394       fprintf                    0000000180002394 f i libIndyRedefineClass.obj
 0001:000013d8       getMethodName              00000001800023d8 f   libIndyRedefineClass.obj
 0001:000015f4       getTLS                     00000001800025f4 f   libIndyRedefineClass.obj
 0001:0000177c       locationToString           000000018000277c f   libIndyRedefineClass.obj
 0001:0000183c       nsk_complain               000000018000283c f   libIndyRedefineClass.obj
 0001:00001868       nsk_jvmti_createJVMTIEnv   0000000180002868 f   libIndyRedefineClass.obj
 0001:00001998       nsk_jvmti_findOptionValue  0000000180002998 f   libIndyRedefineClass.obj
 0001:00001a10       nsk_jvmti_lverify          0000000180002a10 f   libIndyRedefineClass.obj
 0001:00001b00       nsk_jvmti_parseOptions     0000000180002b00 f   libIndyRedefineClass.obj
 0001:00001d50       nsk_jvmti_redefineClass    0000000180002d50 f   libIndyRedefineClass.obj
 0001:00001f60       nsk_jvmti_resetAgentData   0000000180002f60 f   libIndyRedefineClass.obj
 0001:00001fe0       nsk_jvmti_setFailStatus    0000000180002fe0 f   libIndyRedefineClass.obj
 0001:0000201c       nsk_lcomplain              000000018000301c f   libIndyRedefineClass.obj
 0001:0000203c       nsk_ldisplay               000000018000303c f   libIndyRedefineClass.obj
 0001:0000205c       nsk_ltrace                 000000018000305c f   libIndyRedefineClass.obj
 0001:0000207c       nsk_lvcomplain             000000018000307c f   libIndyRedefineClass.obj
 0001:00002234       nsk_lvdisplay              0000000180003234 f   libIndyRedefineClass.obj
 0001:00002280       nsk_lverify                0000000180003280 f   libIndyRedefineClass.obj
 0001:000022dc       nsk_lvtrace                00000001800032dc f   libIndyRedefineClass.obj
 0001:0000233c       nsk_printf                 000000018000333c f   libIndyRedefineClass.obj
 0001:00002364       nsk_vprintf                0000000180003364 f   libIndyRedefineClass.obj
 0001:0000266c       printf                     000000018000366c f i libIndyRedefineClass.obj
 0001:00002b94       __raise_securityfailure    0000000180003b94 f   MSVCRT:gs_report.obj
 0001:00002bc8       __report_gsfailure         0000000180003bc8 f   MSVCRT:gs_report.obj
 0001:00002e08       __GSHandlerCheck           0000000180003e08 f   MSVCRT:gshandler.obj
 0001:00002e28       __GSHandlerCheckCommon     0000000180003e28 f   MSVCRT:gshandler.obj
 0001:00002ea0       __security_check_cookie    0000000180003ea0 f   MSVCRT:amdsecgs.obj
 0001:000031e0       _DllMainCRTStartup         00000001800041e0 f   MSVCRT:dll_dllmain.obj
 0001:00003220       __scrt_acquire_startup_lock 0000000180004220 f   MSVCRT:utility.obj
 0001:0000325c       __scrt_dllmain_after_initialize_c 000000018000425c f   MSVCRT:utility.obj
 0001:00003290       __scrt_dllmain_before_initialize_c 0000000180004290 f   MSVCRT:utility.obj
 0001:000032a8       __scrt_dllmain_crt_thread_attach 00000001800042a8 f   MSVCRT:utility.obj
 0001:000032d0       __scrt_dllmain_crt_thread_detach 00000001800042d0 f   MSVCRT:utility.obj
 0001:000032e8       __scrt_dllmain_exception_filter 00000001800042e8 f   MSVCRT:utility.obj
 0001:00003348       __scrt_dllmain_uninitialize_c 0000000180004348 f   MSVCRT:utility.obj
 0001:00003378       __scrt_dllmain_uninitialize_critical 0000000180004378 f   MSVCRT:utility.obj
 0001:0000338c       __scrt_initialize_crt      000000018000438c f   MSVCRT:utility.obj
 0001:000033d8       __scrt_initialize_onexit_tables 00000001800043d8 f   MSVCRT:utility.obj
 0001:00003464       __scrt_is_nonwritable_in_current_image 0000000180004464 f   MSVCRT:utility.obj
 0001:000034fc       __scrt_release_startup_lock 00000001800044fc f   MSVCRT:utility.obj
 0001:00003520       __scrt_uninitialize_crt    0000000180004520 f   MSVCRT:utility.obj
 0001:0000354c       _onexit                    000000018000454c f   MSVCRT:utility.obj
 0001:00003588       atexit                     0000000180004588 f   MSVCRT:utility.obj
 0001:000035a0       __crt_debugger_hook        00000001800045a0 f   MSVCRT:utility_desktop.obj
 0001:000035a8       __scrt_fastfail            00000001800045a8 f   MSVCRT:utility_desktop.obj
 0001:000036f4       _guard_check_icall_nop     00000001800046f4 f i MSVCRT:guard_support.obj
 0001:000036f8       __security_init_cookie     00000001800046f8 f   MSVCRT:gs_support.obj
 0001:000037a4       DllMain                    00000001800047a4 f   MSVCRT:dll_dllmain_stub.obj
 0001:000037c8       ?__scrt_initialize_type_info@@YAXXZ 00000001800047c8 f   MSVCRT:tncleanup.obj
 0001:000037d8       ?__scrt_uninitialize_type_info@@YAXXZ 00000001800047d8 f   MSVCRT:tncleanup.obj
 0001:000037e4       __local_stdio_scanf_options 00000001800047e4 f i MSVCRT:default_local_stdio_options.obj
 0001:000037ec       __scrt_initialize_default_local_stdio_options 00000001800047ec f   MSVCRT:default_local_stdio_options.obj
 0001:00003808       __scrt_get_dyn_tls_init_callback 0000000180004808 f   MSVCRT:dyn_tls_init.obj
 0001:00003810       _RTC_Initialize            0000000180004810 f   MSVCRT:initsect.obj
 0001:0000384c       _RTC_Terminate             000000018000484c f   MSVCRT:initsect.obj
 0001:00003888       __isa_available_init       0000000180004888 f   MSVCRT:cpu_disp.obj
 0001:00003a34       _get_startup_argv_mode     0000000180004a34 f   MSVCRT:argv_mode.obj
 0001:00003a3c       __scrt_is_ucrt_dll_in_use  0000000180004a3c f   MSVCRT:ucrt_detection.obj
 0001:00003a50       memset                     0000000180004a50 f   vcruntime:VCRUNTIME140.dll
 0001:00003a56       strchr                     0000000180004a56 f   vcruntime:VCRUNTIME140.dll
 0001:00003a5c       __C_specific_handler       0000000180004a5c f   vcruntime:VCRUNTIME140.dll
 0001:00003a62       __std_type_info_destroy_list 0000000180004a62 f   vcruntime:VCRUNTIME140.dll
 0001:00003a68       strcmp                     0000000180004a68 f   ucrt:api-ms-win-crt-string-l1-1-0.dll
 0001:00003a6e       strlen                     0000000180004a6e f   ucrt:api-ms-win-crt-string-l1-1-0.dll
 0001:00003a74       _initterm                  0000000180004a74 f   ucrt:api-ms-win-crt-runtime-l1-1-0.dll
 0001:00003a7a       _initterm_e                0000000180004a7a f   ucrt:api-ms-win-crt-runtime-l1-1-0.dll
 0001:00003a80       _seh_filter_dll            0000000180004a80 f   ucrt:api-ms-win-crt-runtime-l1-1-0.dll
 0001:00003a86       _configure_narrow_argv     0000000180004a86 f   ucrt:api-ms-win-crt-runtime-l1-1-0.dll
 0001:00003a8c       _initialize_narrow_environment 0000000180004a8c f   ucrt:api-ms-win-crt-runtime-l1-1-0.dll
 0001:00003a92       _initialize_onexit_table   0000000180004a92 f   ucrt:api-ms-win-crt-runtime-l1-1-0.dll
 0001:00003a98       _register_onexit_function  0000000180004a98 f   ucrt:api-ms-win-crt-runtime-l1-1-0.dll
 0001:00003a9e       _execute_onexit_table      0000000180004a9e f   ucrt:api-ms-win-crt-runtime-l1-1-0.dll
 0001:00003aa4       _crt_atexit                0000000180004aa4 f   ucrt:api-ms-win-crt-runtime-l1-1-0.dll
 0001:00003aaa       _cexit                     0000000180004aaa f   ucrt:api-ms-win-crt-runtime-l1-1-0.dll
 0001:00003ab0       __acrt_initialize          0000000180004ab0 f   MSVCRT:ucrt_stubs.obj
 0001:00003ab0       __acrt_thread_attach       0000000180004ab0 f   MSVCRT:ucrt_stubs.obj
 0001:00003ab0       __acrt_thread_detach       0000000180004ab0 f   MSVCRT:ucrt_stubs.obj
 0001:00003ab0       __acrt_uninitialize        0000000180004ab0 f   MSVCRT:ucrt_stubs.obj
 0001:00003ab0       __acrt_uninitialize_critical 0000000180004ab0 f   MSVCRT:ucrt_stubs.obj
 0001:00003ab0       __scrt_stub_for_acrt_initialize 0000000180004ab0 f   MSVCRT:ucrt_stubs.obj
 0001:00003ab0       __scrt_stub_for_acrt_thread_attach 0000000180004ab0 f   MSVCRT:ucrt_stubs.obj
 0001:00003ab0       __scrt_stub_for_acrt_thread_detach 0000000180004ab0 f   MSVCRT:ucrt_stubs.obj
 0001:00003ab0       __scrt_stub_for_acrt_uninitialize 0000000180004ab0 f   MSVCRT:ucrt_stubs.obj
 0001:00003ab0       __scrt_stub_for_acrt_uninitialize_critical 0000000180004ab0 f   MSVCRT:ucrt_stubs.obj
 0001:00003ab0       __vcrt_initialize          0000000180004ab0 f   MSVCRT:ucrt_stubs.obj
 0001:00003ab0       __vcrt_thread_attach       0000000180004ab0 f   MSVCRT:ucrt_stubs.obj
 0001:00003ab0       __vcrt_thread_detach       0000000180004ab0 f   MSVCRT:ucrt_stubs.obj
 0001:00003ab0       __vcrt_uninitialize        0000000180004ab0 f   MSVCRT:ucrt_stubs.obj
 0001:00003ab0       __vcrt_uninitialize_critical 0000000180004ab0 f   MSVCRT:ucrt_stubs.obj
 0001:00003ab4       __scrt_stub_for_is_c_termination_complete 0000000180004ab4 f   MSVCRT:ucrt_stubs.obj
 0001:00003ab4       _is_c_termination_complete 0000000180004ab4 f   MSVCRT:ucrt_stubs.obj
 0001:00003ab7       memcpy                     0000000180004ab7 f   vcruntime:VCRUNTIME140.dll
 0001:00003ad0       _guard_dispatch_icall_nop  0000000180004ad0 f   MSVCRT:guard_dispatch.obj
 0001:00003af0       _guard_xfg_dispatch_icall_nop 0000000180004af0 f   MSVCRT:guard_xfg_dispatch.obj
 0002:00000000       __imp_RtlCaptureContext    0000000180005000     kernel32:KERNEL32.dll
 0002:00000008       __imp_RtlLookupFunctionEntry 0000000180005008     kernel32:KERNEL32.dll
 0002:00000010       __imp_RtlVirtualUnwind     0000000180005010     kernel32:KERNEL32.dll
 0002:00000018       __imp_UnhandledExceptionFilter 0000000180005018     kernel32:KERNEL32.dll
 0002:00000020       __imp_SetUnhandledExceptionFilter 0000000180005020     kernel32:KERNEL32.dll
 0002:00000028       __imp_GetCurrentProcess    0000000180005028     kernel32:KERNEL32.dll
 0002:00000030       __imp_TerminateProcess     0000000180005030     kernel32:KERNEL32.dll
 0002:00000038       __imp_IsProcessorFeaturePresent 0000000180005038     kernel32:KERNEL32.dll
 0002:00000040       __imp_CloseHandle          0000000180005040     kernel32:KERNEL32.dll
 0002:00000048       __imp_InitializeCriticalSectionAndSpinCount 0000000180005048     kernel32:KERNEL32.dll
 0002:00000050       __imp_DeleteCriticalSection 0000000180005050     kernel32:KERNEL32.dll
 0002:00000058       __imp_CreateEventW         0000000180005058     kernel32:KERNEL32.dll
 0002:00000060       __imp_GetModuleHandleW     0000000180005060     kernel32:KERNEL32.dll
 0002:00000068       __imp_GetProcAddress       0000000180005068     kernel32:KERNEL32.dll
 0002:00000070       __imp_IsDebuggerPresent    0000000180005070     kernel32:KERNEL32.dll
 0002:00000078       __imp_QueryPerformanceCounter 0000000180005078     kernel32:KERNEL32.dll
 0002:00000080       __imp_GetCurrentProcessId  0000000180005080     kernel32:KERNEL32.dll
 0002:00000088       __imp_GetCurrentThreadId   0000000180005088     kernel32:KERNEL32.dll
 0002:00000090       __imp_GetSystemTimeAsFileTime 0000000180005090     kernel32:KERNEL32.dll
 0002:00000098       __imp_DisableThreadLibraryCalls 0000000180005098     kernel32:KERNEL32.dll
 0002:000000a0       __imp_InitializeSListHead  00000001800050a0     kernel32:KERNEL32.dll
 0002:000000a8       \177KERNEL32_NULL_THUNK_DATA 00000001800050a8     kernel32:KERNEL32.dll
 0002:000000b0       __imp_memset               00000001800050b0     vcruntime:VCRUNTIME140.dll
 0002:000000b8       __imp_strchr               00000001800050b8     vcruntime:VCRUNTIME140.dll
 0002:000000c0       __imp___C_specific_handler 00000001800050c0     vcruntime:VCRUNTIME140.dll
 0002:000000c8       __imp___std_type_info_destroy_list 00000001800050c8     vcruntime:VCRUNTIME140.dll
 0002:000000d0       __imp_memcpy               00000001800050d0     vcruntime:VCRUNTIME140.dll
 0002:000000d8       \177VCRUNTIME140_NULL_THUNK_DATA 00000001800050d8     vcruntime:VCRUNTIME140.dll
 0002:000000e0       __imp_strtol               00000001800050e0     ucrt:api-ms-win-crt-convert-l1-1-0.dll
 0002:000000e8       \177api-ms-win-crt-convert-l1-1-0_NULL_THUNK_DATA 00000001800050e8     ucrt:api-ms-win-crt-convert-l1-1-0.dll
 0002:000000f0       __imp_free                 00000001800050f0     ucrt:api-ms-win-crt-heap-l1-1-0.dll
 0002:000000f8       __imp_malloc               00000001800050f8     ucrt:api-ms-win-crt-heap-l1-1-0.dll
 0002:00000100       \177api-ms-win-crt-heap-l1-1-0_NULL_THUNK_DATA 0000000180005100     ucrt:api-ms-win-crt-heap-l1-1-0.dll
 0002:00000108       __imp__seh_filter_dll      0000000180005108     ucrt:api-ms-win-crt-runtime-l1-1-0.dll
 0002:00000110       __imp__configure_narrow_argv 0000000180005110     ucrt:api-ms-win-crt-runtime-l1-1-0.dll
 0002:00000118       __imp__initterm            0000000180005118     ucrt:api-ms-win-crt-runtime-l1-1-0.dll
 0002:00000120       __imp__initialize_narrow_environment 0000000180005120     ucrt:api-ms-win-crt-runtime-l1-1-0.dll
 0002:00000128       __imp__initialize_onexit_table 0000000180005128     ucrt:api-ms-win-crt-runtime-l1-1-0.dll
 0002:00000130       __imp__register_onexit_function 0000000180005130     ucrt:api-ms-win-crt-runtime-l1-1-0.dll
 0002:00000138       __imp__errno               0000000180005138     ucrt:api-ms-win-crt-runtime-l1-1-0.dll
 0002:00000140       __imp_exit                 0000000180005140     ucrt:api-ms-win-crt-runtime-l1-1-0.dll
 0002:00000148       __imp__execute_onexit_table 0000000180005148     ucrt:api-ms-win-crt-runtime-l1-1-0.dll
 0002:00000150       __imp__crt_atexit          0000000180005150     ucrt:api-ms-win-crt-runtime-l1-1-0.dll
 0002:00000158       __imp__initterm_e          0000000180005158     ucrt:api-ms-win-crt-runtime-l1-1-0.dll
 0002:00000160       __imp__cexit               0000000180005160     ucrt:api-ms-win-crt-runtime-l1-1-0.dll
 0002:00000168       \177api-ms-win-crt-runtime-l1-1-0_NULL_THUNK_DATA 0000000180005168     ucrt:api-ms-win-crt-runtime-l1-1-0.dll
 0002:00000170       __imp_fread                0000000180005170     ucrt:api-ms-win-crt-stdio-l1-1-0.dll
 0002:00000178       __imp___stdio_common_vsprintf 0000000180005178     ucrt:api-ms-win-crt-stdio-l1-1-0.dll
 0002:00000180       __imp___stdio_common_vfprintf 0000000180005180     ucrt:api-ms-win-crt-stdio-l1-1-0.dll
 0002:00000188       __imp_rewind               0000000180005188     ucrt:api-ms-win-crt-stdio-l1-1-0.dll
 0002:00000190       __imp_ftell                0000000180005190     ucrt:api-ms-win-crt-stdio-l1-1-0.dll
 0002:00000198       __imp_fseek                0000000180005198     ucrt:api-ms-win-crt-stdio-l1-1-0.dll
 0002:000001a0       __imp_fopen                00000001800051a0     ucrt:api-ms-win-crt-stdio-l1-1-0.dll
 0002:000001a8       __imp_fflush               00000001800051a8     ucrt:api-ms-win-crt-stdio-l1-1-0.dll
 0002:000001b0       __imp_fclose               00000001800051b0     ucrt:api-ms-win-crt-stdio-l1-1-0.dll
 0002:000001b8       __imp___acrt_iob_func      00000001800051b8     ucrt:api-ms-win-crt-stdio-l1-1-0.dll
 0002:000001c0       \177api-ms-win-crt-stdio-l1-1-0_NULL_THUNK_DATA 00000001800051c0     ucrt:api-ms-win-crt-stdio-l1-1-0.dll
 0002:000001c8       __imp__strdup              00000001800051c8     ucrt:api-ms-win-crt-string-l1-1-0.dll
 0002:000001c8       __imp_strdup               00000001800051c8     ucrt:api-ms-win-crt-string-l1-1-0.dll
 0002:000001d0       __imp_strncpy              00000001800051d0     ucrt:api-ms-win-crt-string-l1-1-0.dll
 0002:000001d8       __imp_strlen               00000001800051d8     ucrt:api-ms-win-crt-string-l1-1-0.dll
 0002:000001e0       __imp_strcmp               00000001800051e0     ucrt:api-ms-win-crt-string-l1-1-0.dll
 0002:000001e8       __imp_strpbrk              00000001800051e8     ucrt:api-ms-win-crt-string-l1-1-0.dll
 0002:000001f0       \177api-ms-win-crt-string-l1-1-0_NULL_THUNK_DATA 00000001800051f0     ucrt:api-ms-win-crt-string-l1-1-0.dll
 0002:000001f8       __guard_check_icall_fptr   00000001800051f8     MSVCRT:guard_support.obj
 0002:00000200       __guard_xfg_check_icall_fptr 0000000180005200     MSVCRT:guard_support.obj
 0002:00000208       __guard_dispatch_icall_fptr 0000000180005208     MSVCRT:guard_support.obj
 0002:00000210       __guard_xfg_dispatch_icall_fptr 0000000180005210     MSVCRT:guard_support.obj
 0002:00000218       __guard_xfg_table_dispatch_icall_fptr 0000000180005218     MSVCRT:guard_support.obj
 0002:00000220       __castguard_check_failure_os_handled_fptr 0000000180005220     MSVCRT:guard_support.obj
 0002:00000228       __guard_memcpy_fptr        0000000180005228     vcruntime:softmemtag.obj
 0002:00000230       __xc_a                     0000000180005230     MSVCRT:initializers.obj
 0002:00000238       __xc_z                     0000000180005238     MSVCRT:initializers.obj
 0002:00000240       __xi_a                     0000000180005240     MSVCRT:initializers.obj
 0002:00000250       __xi_z                     0000000180005250     MSVCRT:initializers.obj
 0002:00000258       __xl_a                     0000000180005258     MSVCRT:tlssup.obj
 0002:00000260       __xl_z                     0000000180005260     MSVCRT:tlssup.obj
 0002:00000268       __xp_a                     0000000180005268     MSVCRT:initializers.obj
 0002:00000270       __xp_z                     0000000180005270     MSVCRT:initializers.obj
 0002:00000278       __xt_a                     0000000180005278     MSVCRT:initializers.obj
 0002:00000280       __xt_z                     0000000180005280     MSVCRT:initializers.obj
 0002:00000290       ??_C@_04OKGDLNCL@NONE@     0000000180005290     libIndyRedefineClass.obj
 0002:00000298       ??_C@_0BB@JCNMKLLK@JVMTI_ERROR_NONE@ 0000000180005298     libIndyRedefineClass.obj
 0002:000002b0       ??_C@_0BL@LDIMKLPH@JVMTI_ERROR_INVALID_THREAD@ 00000001800052b0     libIndyRedefineClass.obj
 0002:000002d0       ??_C@_0CB@PJFPAIKJ@JVMTI_ERROR_INVALID_THREAD_GROU@ 00000001800052d0     libIndyRedefineClass.obj
 0002:000002f8       ??_C@_0BN@LLMKHMNF@JVMTI_ERROR_INVALID_PRIORITY@ 00000001800052f8     libIndyRedefineClass.obj
 0002:00000318       ??_C@_0CB@MBOFKAGB@JVMTI_ERROR_THREAD_NOT_SUSPENDE@ 0000000180005318     libIndyRedefineClass.obj
 0002:00000340       ??_C@_0BN@FABOLPBI@JVMTI_ERROR_THREAD_SUSPENDED@ 0000000180005340     libIndyRedefineClass.obj
 0002:00000360       ??_C@_0BN@FDGNOBJM@JVMTI_ERROR_THREAD_NOT_ALIVE@ 0000000180005360     libIndyRedefineClass.obj
 0002:00000380       ??_C@_0BL@GOBIFKNJ@JVMTI_ERROR_INVALID_OBJECT@ 0000000180005380     libIndyRedefineClass.obj
 0002:000003a0       ??_C@_0BK@FCMAJPPC@JVMTI_ERROR_INVALID_CLASS@ 00000001800053a0     libIndyRedefineClass.obj
 0002:000003c0       ??_C@_0BP@IKLLBKEB@JVMTI_ERROR_CLASS_NOT_PREPARED@ 00000001800053c0     libIndyRedefineClass.obj
 0002:000003e0       ??_C@_0BN@KLPPLKG@JVMTI_ERROR_INVALID_METHODID@ 00000001800053e0     libIndyRedefineClass.obj
 0002:00000400       ??_C@_0BN@BCEKOKND@JVMTI_ERROR_INVALID_LOCATION@ 0000000180005400     libIndyRedefineClass.obj
 0002:00000420       ??_C@_0BM@DFDGPME@JVMTI_ERROR_INVALID_FIELDID@ 0000000180005420     libIndyRedefineClass.obj
 0002:00000440       ??_C@_0BL@NELIEPEC@JVMTI_ERROR_NO_MORE_FRAMES@ 0000000180005440     libIndyRedefineClass.obj
 0002:00000460       ??_C@_0BJ@BDBECFDM@JVMTI_ERROR_OPAQUE_FRAME@ 0000000180005460     libIndyRedefineClass.obj
 0002:00000480       ??_C@_0BK@MIIFNLOB@JVMTI_ERROR_TYPE_MISMATCH@ 0000000180005480     libIndyRedefineClass.obj
 0002:000004a0       ??_C@_0BJ@HPCAOILC@JVMTI_ERROR_INVALID_SLOT@ 00000001800054a0     libIndyRedefineClass.obj
 0002:000004c0       ??_C@_0BG@CHILOPNI@JVMTI_ERROR_DUPLICATE@ 00000001800054c0     libIndyRedefineClass.obj
 0002:000004d8       ??_C@_0BG@DIEMLHKM@JVMTI_ERROR_NOT_FOUND@ 00000001800054d8     libIndyRedefineClass.obj
 0002:000004f0       ??_C@_0BM@NHMCKHOB@JVMTI_ERROR_INVALID_MONITOR@ 00000001800054f0     libIndyRedefineClass.obj
 0002:00000510       ??_C@_0BO@PPEDAJGL@JVMTI_ERROR_NOT_MONITOR_OWNER@ 0000000180005510     libIndyRedefineClass.obj
 0002:00000530       ??_C@_0BG@FCAIPEID@JVMTI_ERROR_INTERRUPT@ 0000000180005530     libIndyRedefineClass.obj
 0002:00000548       ??_C@_0CB@EGDBNKOI@JVMTI_ERROR_INVALID_CLASS_FORMA@ 0000000180005548     libIndyRedefineClass.obj
 0002:00000570       ??_C@_0CG@DGKOGIAL@JVMTI_ERROR_CIRCULAR_CLASS_DEFI@ 0000000180005570     libIndyRedefineClass.obj
 0002:00000598       ??_C@_0BP@ICEALPKC@JVMTI_ERROR_FAILS_VERIFICATION@ 0000000180005598     libIndyRedefineClass.obj
 0002:000005b8       ??_C@_0DC@JDACLMIO@JVMTI_ERROR_UNSUPPORTED_REDEFIN@ 00000001800055b8     libIndyRedefineClass.obj
 0002:000005f0       ??_C@_0DE@GKDKNOMJ@JVMTI_ERROR_UNSUPPORTED_REDEFIN@ 00000001800055f0     libIndyRedefineClass.obj
 0002:00000628       ??_C@_0BO@LAFKIOG@JVMTI_ERROR_INVALID_TYPESTATE@ 0000000180005628     libIndyRedefineClass.obj
 0002:00000648       ??_C@_0DH@INDGCLLB@JVMTI_ERROR_UNSUPPORTED_REDEFIN@ 0000000180005648     libIndyRedefineClass.obj
 0002:00000680       ??_C@_0DE@NHEOMMGI@JVMTI_ERROR_UNSUPPORTED_REDEFIN@ 0000000180005680     libIndyRedefineClass.obj
 0002:000006b8       ??_C@_0CA@EKPNJOEP@JVMTI_ERROR_UNSUPPORTED_VERSION@ 00000001800056b8     libIndyRedefineClass.obj
 0002:000006d8       ??_C@_0BN@OFFMAHHL@JVMTI_ERROR_NAMES_DONT_MATCH@ 00000001800056d8     libIndyRedefineClass.obj
 0002:000006f8       ??_C@_0DN@HHBBLAKE@JVMTI_ERROR_UNSUPPORTED_REDEFIN@ 00000001800056f8     libIndyRedefineClass.obj
 0002:00000738       ??_C@_0DO@HMBGBGNA@JVMTI_ERROR_UNSUPPORTED_REDEFIN@ 0000000180005738     libIndyRedefineClass.obj
 0002:00000778       ??_C@_0BP@PBECGKHJ@JVMTI_ERROR_UNMODIFIABLE_CLASS@ 0000000180005778     libIndyRedefineClass.obj
 0002:00000798       ??_C@_0BK@CANILEHF@JVMTI_ERROR_NOT_AVAILABLE@ 0000000180005798     libIndyRedefineClass.obj
 0002:000007b8       ??_C@_0CE@INJKMEFK@JVMTI_ERROR_MUST_POSSESS_CAPABI@ 00000001800057b8     libIndyRedefineClass.obj
 0002:000007e0       ??_C@_0BJ@LBFPFPDM@JVMTI_ERROR_NULL_POINTER@ 00000001800057e0     libIndyRedefineClass.obj
 0002:00000800       ??_C@_0BP@CHJPNNEM@JVMTI_ERROR_ABSENT_INFORMATION@ 0000000180005800     libIndyRedefineClass.obj
 0002:00000820       ??_C@_0BP@OMFMNLC@JVMTI_ERROR_INVALID_EVENT_TYPE@ 0000000180005820     libIndyRedefineClass.obj
 0002:00000840       ??_C@_0BN@BIBNPHHO@JVMTI_ERROR_ILLEGAL_ARGUMENT@ 0000000180005840     libIndyRedefineClass.obj
 0002:00000860       ??_C@_0BK@KKNDHDCE@JVMTI_ERROR_NATIVE_METHOD@ 0000000180005860     libIndyRedefineClass.obj
 0002:00000880       ??_C@_0BK@PMKCFHAE@JVMTI_ERROR_OUT_OF_MEMORY@ 0000000180005880     libIndyRedefineClass.obj
 0002:000008a0       ??_C@_0BK@NNJBDMNB@JVMTI_ERROR_ACCESS_DENIED@ 00000001800058a0     libIndyRedefineClass.obj
 0002:000008c0       ??_C@_0BI@GHECLMNC@JVMTI_ERROR_WRONG_PHASE@ 00000001800058c0     libIndyRedefineClass.obj
 0002:000008d8       ??_C@_0BF@OLIHJOII@JVMTI_ERROR_INTERNAL@ 00000001800058d8     libIndyRedefineClass.obj
 0002:000008f0       ??_C@_0BO@EOHGKJHI@JVMTI_ERROR_UNATTACHED_THREAD@ 00000001800058f0     libIndyRedefineClass.obj
 0002:00000910       ??_C@_0CA@LKHFDACL@JVMTI_ERROR_INVALID_ENVIRONMENT@ 0000000180005910     libIndyRedefineClass.obj
 0002:00000930       ??_C@_0BA@MMFHLOKK@?$DMunknown?5error?$DO@ 0000000180005930     libIndyRedefineClass.obj
 0002:00000940       ??_C@_0L@HCDIAMJG@?9?5?$CFs?0?5?$CFd?3?5@ 0000000180005940     libIndyRedefineClass.obj
 0002:00000950       ??_C@_0JI@HLPECLFI@?$CD?5?4?4?4?6?$CD?5ERROR?3?5too?5many?5complai@ 0000000180005950     libIndyRedefineClass.obj
 0002:000009f0       ??_C@_0ED@JNEKCCOB@The?5following?5fake?5exception?5st@ 00000001800059f0     libIndyRedefineClass.obj
 0002:00000a38       ??_C@_0CN@FCNMDFBH@nsk?4share?4Fake_Exception_for_RU@ 0000000180005a38     libIndyRedefineClass.obj
 0002:00000a68       ??_C@_08PGFFNAEI@?$CI?$CFs?3?$CFd?$CJ?5@ 0000000180005a68     libIndyRedefineClass.obj
 0002:00000a78       ??_C@_0DP@IENMAEGI@s?2test?2hotspot?2jtreg?2vmTestbase@ 0000000180005a78     libIndyRedefineClass.obj
 0002:00000ab8       ??_C@_0BL@NDJLFFJB@?7at?5nsk_lvcomplain?$CI?$CFs?3?$CFd?$CJ?6@ 0000000180005ab8     libIndyRedefineClass.obj
 0002:00000ad8       ??_C@_0BC@JOOKAFKF@?$CD?5ERROR?3?5?$CFs?0?5?$CFd?3?5@ 0000000180005ad8     libIndyRedefineClass.obj
 0002:00000af0       ??_C@_09KJEAHMEH@?$CD?5ERROR?3?5@ 0000000180005af0     libIndyRedefineClass.obj
 0002:00000afc       ??_C@_02GPIOPFAK@?$DO?$DO@ 0000000180005afc     libIndyRedefineClass.obj
 0002:00000b00       ??_C@_02FODMEDOG@?$DM?$DM@ 0000000180005b00     libIndyRedefineClass.obj
 0002:00000b04       ??_C@_02DJGKEECL@?4?4@     0000000180005b04     libIndyRedefineClass.obj
 0002:00000b08       ??_C@_0O@CJPGJOAF@?9?5?$CFs?0?5?$CFd?3?5?$CFs?5@ 0000000180005b08     libIndyRedefineClass.obj
 0002:00000b18       ??_C@_0CB@IAKPDOIC@?$CD?5?5?5verified?5assertion?5is?5FALSE@ 0000000180005b18     libIndyRedefineClass.obj
 0002:00000b40       ??_C@_0CO@LGONDEPD@stdout?3?5fflush?5failed?5?9?5err?$DN?$CFd?5@ 0000000180005b40     libIndyRedefineClass.obj
 0002:00000b70       ??_C@_0CO@KBGKJPBD@stderr?3?5fflush?5failed?5?9?5err?$DN?$CFd?5@ 0000000180005b70     libIndyRedefineClass.obj
 0002:00000ba0       ??_C@_0CF@CBHOKDB@throwable?5?$DN?5jni?9?$DOExceptionOccur@ 0000000180005ba0     libIndyRedefineClass.obj
 0002:00000bc8       ??_C@_03OFAPEBGM@?$CFs?6@  0000000180005bc8     libIndyRedefineClass.obj
 0002:00000bd0       ??_C@_0DM@LPIGEGNJ@s?2test?2hotspot?2jtreg?2vmTestbase@ 0000000180005bd0     libIndyRedefineClass.obj
 0002:00000c10       ??_C@_0CC@NFCNPEPK@Exception?5in?5JNI?5call?5?$CIcleared?$CJ@ 0000000180005c10     libIndyRedefineClass.obj
 0002:00000c38       ??_C@_0BJ@IBAKFIKF@jni?9?$DOExceptionDescribe?$CI?$CJ@ 0000000180005c38     libIndyRedefineClass.obj
 0002:00000c58       ??_C@_0BG@GGKALKMH@jni?9?$DOExceptionClear?$CI?$CJ@ 0000000180005c58     libIndyRedefineClass.obj
 0002:00000c70       ??_C@_0CF@JMGFGJLJ@?$CD?5?5?5verified?5JNI?5assertion?5is?5F@ 0000000180005c70     libIndyRedefineClass.obj
 0002:00000c98       ??_C@_0CJ@JACLEAA@Test?5failed?5by?5setFailStatus?$CI?$CJ?4@ 0000000180005c98     libIndyRedefineClass.obj
 0002:00000cc8       ??_C@_0BD@HGNAOMCP@agent_data_monitor@ 0000000180005cc8     libIndyRedefineClass.obj
 0002:00000ce0       ??_C@_0EB@OGCLGKLN@javaVM?9?$DOGetEnv?$CI?$CIvoid?5?$CK?$CK?$CJ?$CGjvmti_@ 0000000180005ce0     libIndyRedefineClass.obj
 0002:00000d30       ??_C@_0EA@PNBCDMOA@s?2test?2hotspot?2jtreg?2vmTestbase@ 0000000180005d30     libIndyRedefineClass.obj
 0002:00000d70       ??_C@_0CI@DDPIFBGM@init_agent_data?$CIjvmti_env?0?5?$CGage@ 0000000180005d70     libIndyRedefineClass.obj
 0002:00000d98       ??_C@_0DI@ILAHDLMP@?$CI?$CKagentThreadProc?$CJ?$CIjvmti_env?0?5a@ 0000000180005d98     libIndyRedefineClass.obj
 0002:00000dd0       ??_C@_0BD@KDBALNLB@JVMTI?5agent?5thread@ 0000000180005dd0     libIndyRedefineClass.obj
 0002:00000de8       ??_C@_0BB@NOKBFPFO@java?1lang?1Thread@ 0000000180005de8     libIndyRedefineClass.obj
 0002:00000dfc       ??_C@_06FALKBLGB@?$DMinit?$DO@ 0000000180005dfc     libIndyRedefineClass.obj
 0002:00000e08       ??_C@_0BG@IKDDPPGD@?$CILjava?1lang?1String?$DL?$CJV@ 0000000180005e08     libIndyRedefineClass.obj
 0002:00000e20       ??_C@_0EB@IFJBFEKC@?$CIthreadClass?5?$DN?5jni_env?9?$DOFindCla@ 0000000180005e20     libIndyRedefineClass.obj
 0002:00000e70       ??_C@_0GF@FGFIBKKL@?$CIthreadCtor?5?$DN?5jni_env?9?$DOGetMetho@ 0000000180005e70     libIndyRedefineClass.obj
 0002:00000ed8       ??_C@_0DN@NCPDJLOG@?$CIthreadName?5?$DN?5jni_env?9?$DONewStrin@ 0000000180005ed8     libIndyRedefineClass.obj
 0002:00000f20       ??_C@_0FE@PFKODBGC@?$CIthreadObject?5?$DN?5jni_env?9?$DONewObj@ 0000000180005f20     libIndyRedefineClass.obj
 0002:00000f80       ??_C@_0ED@HOBAHHJI@?$CIthreadGlobalRef?5?$DN?5jni_env?9?$DONew@ 0000000180005f80     libIndyRedefineClass.obj
 0002:00000fd0       ??_C@_0FN@HNJJAHFC@jvmti_env?9?$DORunAgentThread?$CIagent@ 0000000180005fd0     libIndyRedefineClass.obj
 0002:00001030       ??_C@_0EA@MOJDNKDF@Debuggee?5status?5sync?5aborted?5be@ 0000000180006030     libIndyRedefineClass.obj
 0002:00001070       ??_C@_0EA@EEOEJAEN@status?5?$DN?5syncDebuggeeStatus?$CIjni@ 0000000180006070     libIndyRedefineClass.obj
 0002:000010b0       ??_C@_0BL@JBCFNBMB@nsk_jvmti_resetAgentData?$CI?$CJ@ 00000001800060b0     libIndyRedefineClass.obj
 0002:000010d0       ??_C@_07KBAMPNJK@verbose@  00000001800060d0     libIndyRedefineClass.obj
 0002:000010d8       ??_C@_0DN@PKJBOLAP@nsk_jvmti_parseOptions?$CI?$CJ?3?5unexp@ 00000001800060d8     libIndyRedefineClass.obj
 0002:00001118       ??_C@_05IMBNNINJ@trace@    0000000180006118     libIndyRedefineClass.obj
 0002:00001120       ??_C@_0DD@BJKGNDMB@nsk_jvmti_parseOptions?$CI?$CJ?3?5no?5va@ 0000000180006120     libIndyRedefineClass.obj
 0002:00001154       ??_C@_04CGFJFPFD@none@     0000000180006154     libIndyRedefineClass.obj
 0002:0000115c       ??_C@_06BMELKFMA@before@   000000018000615c     libIndyRedefineClass.obj
 0002:00001164       ??_C@_05CMKPCFDK@after@    0000000180006164     libIndyRedefineClass.obj
 0002:0000116c       ??_C@_03NFKEKGGK@all@      000000018000616c     libIndyRedefineClass.obj
 0002:00001170       ??_C@_0DM@NDNJGJKE@nsk_jvmti_parseOptions?$CI?$CJ?3?5uexpe@ 0000000180006170     libIndyRedefineClass.obj
 0002:000011b0       ??_C@_08NBBJKJO@waittime@  00000001800061b0     libIndyRedefineClass.obj
 0002:000011c0       ??_C@_0DO@CMHGAOHC@nsk_jvmti_parseOptions?$CI?$CJ?3?5not?5i@ 00000001800061c0     libIndyRedefineClass.obj
 0002:00001200       ??_C@_0DL@LNMPBDLN@nsk_jvmti_parseOptions?$CI?$CJ?3?5negat@ 0000000180006200     libIndyRedefineClass.obj
 0002:00001240       ??_C@_0DA@GMFJNOJH@nsk_jvmti_parseOptions?$CI?$CJ?3?5unkno@ 0000000180006240     libIndyRedefineClass.obj
 0002:00001270       ??_C@_0CO@CCIAMEAN@nsk_jvmti_parseOptions?$CI?$CJ?3?5found@ 0000000180006270     libIndyRedefineClass.obj
 0002:000012a0       ??_C@_0CJ@OEGPCGDL@nsk_jvmti_parseOptions?$CI?$CJ?3?5out?5o@ 00000001800062a0     libIndyRedefineClass.obj
 0002:000012d0       ??_C@_0DI@NMBHPGGF@nsk_jvmti_parseOptions?$CI?$CJ?3?5too?5m@ 00000001800062d0     libIndyRedefineClass.obj
 0002:00001308       ??_C@_03POGCGECB@?5?0?$HO@ 0000000180006308     libIndyRedefineClass.obj
 0002:00001310       ??_C@_0DC@GKLNPJIJ@nsk_jvmti_findOptionValue?$CI?$CJ?3?5op@ 0000000180006310     libIndyRedefineClass.obj
 0002:00001348       ??_C@_0CB@MLNJNCLJ@?5?5jvmti?5error?3?5code?$DN?$CFd?0?5name?$DN?$CFs@ 0000000180006348     libIndyRedefineClass.obj
 0002:00001370       ??_C@_0CD@OHBGDKMK@?$CD?5?5?5jvmti?5error?3?5code?$DN?$CFd?0?5name?$DN@ 0000000180006370     libIndyRedefineClass.obj
 0002:00001398       ??_C@_0CG@JNNCGPHB@?$CD?5?5?5error?5expected?3?5code?$DN?$CFd?0?5na@ 0000000180006398     libIndyRedefineClass.obj
 0002:000013c0       ??_C@_0EB@IMGKPCGE@?$CIstr_obj?5?$DN?5jni?9?$DONewStringUTF?$CIco@ 00000001800063c0     libIndyRedefineClass.obj
 0002:00001410       ??_C@_0EA@HFOGGBCC@s?2test?2hotspot?2jtreg?2vmTestbase@ 0000000180006410     libIndyRedefineClass.obj
 0002:00001450       ??_C@_0BC@PAGIDHOM@pathToNewByteCode@ 0000000180006450     libIndyRedefineClass.obj
 0002:00001468       ??_C@_0BJ@NJNNDFOA@?$CD?5?5?5error?5expected?3?5?$CFs?5?6@ 0000000180006468     libIndyRedefineClass.obj
 0002:00001490       ??_C@_0EG@ELLMOONO@Hint?5?3?3?5missing?5java?5?9agentlib?3@ 0000000180006490     libIndyRedefineClass.obj
 0002:000014d8       ??_C@_0CL@NDJEIHKI@?$CD?5error?5file?5name?5expected?5did?5@ 00000001800064d8     libIndyRedefineClass.obj
 0002:00001508       ??_C@_0M@KLIIGBGL@?$CFs?1?$CFs?4class@ 0000000180006508     libIndyRedefineClass.obj
 0002:00001518       ??_C@_0BG@NPOHJPEP@?$CD?5info?5?3?3?5File?5?$DN?5?$CFs?5?6@ 0000000180006518     libIndyRedefineClass.obj
 0002:00001530       ??_C@_02JDPG@rb@           0000000180006530     libIndyRedefineClass.obj
 0002:00001538       ??_C@_0CJ@MNPKBKGK@?$CD?5error?5?$CK?$CKAgent?3?3error?5opening?5@ 0000000180006538     libIndyRedefineClass.obj
 0002:00001568       ??_C@_0CE@GCANLHLE@?$CD?5?5info?5?$CK?$CKAgent?3?3?5opening?5file?5@ 0000000180006568     libIndyRedefineClass.obj
 0002:00001590       ??_C@_0BH@BAGPKOBE@?$CD?5info?5file?5size?$DN?5?$CFld?6@ 0000000180006590     libIndyRedefineClass.obj
 0002:000015a8       ??_C@_0BO@HAFCJEDK@?5Failed?5to?5create?5memory?5?$CFs?5?6@ 00000001800065a8     libIndyRedefineClass.obj
 0002:000015d0       ??_C@_0EA@BFGBADHF@?5?$CD?5error?5failed?5to?5read?5all?5the@ 00000001800065d0     libIndyRedefineClass.obj
 0002:00001610       ??_C@_0BH@ICCDAOFI@?5File?5red?5completely?5?6@ 0000000180006610     libIndyRedefineClass.obj
 0002:00001628       ??_C@_0CF@OKNNGJPG@?$CD?5error?5occured?5while?5redefinin@ 0000000180006628     libIndyRedefineClass.obj
 0002:00001650       ??_C@_05KKCIMGE@error@     0000000180006650     libIndyRedefineClass.obj
 0002:00001658       ??_C@_0DK@ECIONNCC@?$CIpStr?5?$DN?5pEnv?9?$DOGetStringUTFChars@ 0000000180006658     libIndyRedefineClass.obj
 0002:000016a0       ??_C@_0EB@IJADDDH@s?2test?2hotspot?2jtreg?2vmTestbase@ 00000001800066a0     libIndyRedefineClass.obj
 0002:000016e8       ??_C@_0CM@OCAONMAM@_jvmtiEnv?9?$DODeallocate?$CI?$CIunsigned@ 00000001800066e8     libIndyRedefineClass.obj
 0002:00001718       ??_C@_0DM@KEPBLLAH@pJvmtiEnv?9?$DOGetMethodName?$CImethod@ 0000000180006718     libIndyRedefineClass.obj
 0002:00001758       ??_C@_0DD@BLAEMAPC@pJvmtiEnv?9?$DOGetMethodDeclaringCl@ 0000000180006758     libIndyRedefineClass.obj
 0002:00001790       ??_C@_0DL@IAICHCNL@pJvmtiEnv?9?$DOGetClassSignature?$CIcl@ 0000000180006790     libIndyRedefineClass.obj
 0002:000017d0       ??_C@_0N@GCGOJGML@?$CFs?5?4?$CFs?5?3?$CFlld@ 00000001800067d0     libIndyRedefineClass.obj
 0002:000017e0       ??_C@_0CP@CDOLGEPD@pJvmtiEnv?9?$DOGetThreadLocalStorag@ 00000001800067e0     libIndyRedefineClass.obj
 0002:00001810       ??_C@_0CK@ELKGOPIB@?$CItls?5?$DN?5malloc?$CIsizeToAllocate?$CJ?$CJ?5@ 0000000180006810     libIndyRedefineClass.obj
 0002:00001840       ??_C@_0CO@DHIBHBDK@pJvmtiEnv?9?$DOSetThreadLocalStorag@ 0000000180006840     libIndyRedefineClass.obj
 0002:00001870       ??_C@_0CM@OBPIHPHL@Setting?5redefine?5trigger?5method@ 0000000180006870     libIndyRedefineClass.obj
 0002:000018a0       ??_C@_0FE@EOGCLKHG@s?2test?2hotspot?2jtreg?2vmTestbase@ 00000001800068a0     libIndyRedefineClass.obj
 0002:000018f8       ??_C@_0CE@CMOMBHGK@Setting?5redefined?5class?5name?5to@ 00000001800068f8     libIndyRedefineClass.obj
 0002:00001920       ??_C@_0DL@NIMOFHBP@The?5following?5values?5should?5be?5@ 0000000180006920     libIndyRedefineClass.obj
 0002:00001960       ??_C@_0BO@OIOJJPFO@Method?5entry?5event?5fired?$DP?5?$CFi?6@ 0000000180006960     libIndyRedefineClass.obj
 0002:00001980       ??_C@_0BN@MPKLCJLH@Single?5step?5event?5fired?$DP?5?$CFi?6@ 0000000180006980     libIndyRedefineClass.obj
 0002:000019a0       ??_C@_0DG@LMFJOBJF@The?5following?5value?5should?5be?5z@ 00000001800069a0     libIndyRedefineClass.obj
 0002:000019d8       ??_C@_0BN@FLFOCAGK@Any?5other?5error?5occured?$DP?5?$CFi?6@ 00000001800069d8     libIndyRedefineClass.obj
 0002:000019f8       ??_C@_0BH@MLLNKLHE@Disabling?5single?5step?6@ 00000001800069f8     libIndyRedefineClass.obj
 0002:00001a10       ??_C@_0FF@DLNCHFCG@jvmti_env?9?$DOSetEventNotification@ 0000000180006a10     libIndyRedefineClass.obj
 0002:00001a68       ??_C@_0BG@JKOKDNAP@Enabling?5single?5step?6@ 0000000180006a68     libIndyRedefineClass.obj
 0002:00001a80       ??_C@_0FE@CGHKEFAA@jvmti_env?9?$DOSetEventNotification@ 0000000180006a80     libIndyRedefineClass.obj
 0002:00001ad8       ??_C@_0BB@JMCHCMJC@Popping?5a?5frame?6@ 0000000180006ad8     libIndyRedefineClass.obj
 0002:00001af0       ??_C@_0BM@GMFCOCOP@jvmti_env?9?$DOPopFrame?$CIthread?$CJ@ 0000000180006af0     libIndyRedefineClass.obj
 0002:00001b10       ??_C@_0BG@ECBELDLN@Forcing?5early?5return?6@ 0000000180006b10     libIndyRedefineClass.obj
 0002:00001b28       ??_C@_0CI@GCJIPGG@jvmti_env?9?$DOForceEarlyReturnVoid@ 0000000180006b28     libIndyRedefineClass.obj
 0002:00001b50       ??_C@_0CI@GIJNHBNG@Entering?5redefine?5tigger?5method@ 0000000180006b50     libIndyRedefineClass.obj
 0002:00001b78       ??_C@_0BN@EHDDMLOB@Class?5is?5already?5redefined?4?6@ 0000000180006b78     libIndyRedefineClass.obj
 0002:00001b98       ??_C@_0BF@MFIKHONF@Redefining?5class?5?$CFs?6@ 0000000180006b98     libIndyRedefineClass.obj
 0002:00001bb0       ??_C@_0DD@ENGJGINA@jvmti_env?9?$DOGetMethodDeclaringCl@ 0000000180006bb0     libIndyRedefineClass.obj
 0002:00001bf0       ??_C@_0EF@PGGLHLMH@nsk_jvmti_redefineClass?$CIjvmti_e@ 0000000180006bf0     libIndyRedefineClass.obj
 0002:00001c38       ??_C@_0DF@FODKCKNP@Error?5in?5Single?5step?5event?3?5loc@ 0000000180006c38     libIndyRedefineClass.obj
 0002:00001c70       ??_C@_0BH@FFAOHEJM@Single?5step?5event?3?5?$CFs?6@ 0000000180006c70     libIndyRedefineClass.obj
 0002:00001c88       ??_C@_0CA@MNKGCBCG@nsk_jvmti_parseOptions?$CIoptions?$CJ@ 0000000180006c88     libIndyRedefineClass.obj
 0002:00001cb0       ??_C@_0EA@IGPPECPI@?$CIgJvmtiEnv?5?$DN?5nsk_jvmti_createJV@ 0000000180006cb0     libIndyRedefineClass.obj
 0002:00001cf0       ??_C@_0BD@MCEEOAON@debuggerCompatible@ 0000000180006cf0     libIndyRedefineClass.obj
 0002:00001d08       ??_C@_0CC@JFNNIPAB@gJvmtiEnv?9?$DOAddCapabilities?$CI?$CGcap@ 0000000180006d08     libIndyRedefineClass.obj
 0002:00001d30       ??_C@_0DM@ELBMHCOI@gJvmtiEnv?9?$DOSetEventCallbacks?$CI?$CGc@ 0000000180006d30     libIndyRedefineClass.obj
 0002:00001d70       ??_C@_0FF@FKLNHJHB@gJvmtiEnv?9?$DOSetEventNotification@ 0000000180006d70     libIndyRedefineClass.obj
 0002:00001dd0       ??_C@_0FF@CEGIDDCE@gJvmtiEnv?9?$DOSetEventNotification@ 0000000180006dd0     libIndyRedefineClass.obj
 0002:00001e40       ??_C@_1EC@JIJBPKFM@?$AAa?$AAp?$AAi?$AA?9?$AAm?$AAs?$AA?9?$AAw?$AAi?$AAn?$AA?9?$AAc?$AAo?$AAr?$AAe@ 0000000180006e40     MSVCRT:thread_safe_statics.obj
 0002:00001e88       ??_C@_1BK@MGMFAEKH@?$AAk?$AAe?$AAr?$AAn?$AAe?$AAl?$AA3?$AA2?$AA?4?$AAd?$AAl?$AAl@ 0000000180006e88     MSVCRT:thread_safe_statics.obj
 0002:00001ea8       ??_C@_0BJ@JEBJOJFJ@SleepConditionVariableCS@ 0000000180006ea8     MSVCRT:thread_safe_statics.obj
 0002:00001ec8       ??_C@_0BJ@PGPPEPCC@WakeAllConditionVariable@ 0000000180006ec8     MSVCRT:thread_safe_statics.obj
 0002:00001ee8       _pDefaultRawDllMain        0000000180006ee8     MSVCRT:dll_dllmain.obj
 0002:00001ee8       _pRawDllMain               0000000180006ee8     MSVCRT:dll_dllmain.obj
 0002:00001ef0       __xmm@ffffffffffffffffffffffffffffffff 0000000180006ef0     MSVCRT:utility.obj
 0002:00001f00       _load_config_used          0000000180006f00     MSVCRT:loadcfg.obj
 0002:00002100       _tls_used                  0000000180007100     MSVCRT:tlssup.obj
 0002:00002128       __volatile_metadata        0000000180007128     <linker-defined>
 0002:000024f8       __rtc_iaa                  00000001800074f8     MSVCRT:initsect.obj
 0002:00002500       __rtc_izz                  0000000180007500     MSVCRT:initsect.obj
 0002:00002508       __rtc_taa                  0000000180007508     MSVCRT:initsect.obj
 0002:00002510       __rtc_tzz                  0000000180007510     MSVCRT:initsect.obj
 0002:00002518       _tls_start                 0000000180007518     MSVCRT:tlssup.obj
 0002:0000251c       _Init_thread_epoch         000000018000751c     MSVCRT:thread_safe_statics.obj
 0002:00002520       _tls_end                   0000000180007520     MSVCRT:tlssup.obj
 0002:00002c30       __IMPORT_DESCRIPTOR_KERNEL32 0000000180007c30     kernel32:KERNEL32.dll
 0002:00002c44       __IMPORT_DESCRIPTOR_VCRUNTIME140 0000000180007c44     vcruntime:VCRUNTIME140.dll
 0002:00002c58       __IMPORT_DESCRIPTOR_api-ms-win-crt-stdio-l1-1-0 0000000180007c58     ucrt:api-ms-win-crt-stdio-l1-1-0.dll
 0002:00002c6c       __IMPORT_DESCRIPTOR_api-ms-win-crt-runtime-l1-1-0 0000000180007c6c     ucrt:api-ms-win-crt-runtime-l1-1-0.dll
 0002:00002c80       __IMPORT_DESCRIPTOR_api-ms-win-crt-heap-l1-1-0 0000000180007c80     ucrt:api-ms-win-crt-heap-l1-1-0.dll
 0002:00002c94       __IMPORT_DESCRIPTOR_api-ms-win-crt-convert-l1-1-0 0000000180007c94     ucrt:api-ms-win-crt-convert-l1-1-0.dll
 0002:00002ca8       __IMPORT_DESCRIPTOR_api-ms-win-crt-string-l1-1-0 0000000180007ca8     ucrt:api-ms-win-crt-string-l1-1-0.dll
 0002:00002cbc       __NULL_IMPORT_DESCRIPTOR   0000000180007cbc     kernel32:KERNEL32.dll
 0003:00000018       _Init_global_epoch         0000000180009018     MSVCRT:thread_safe_statics.obj
 0003:00000020       __security_cookie          0000000180009020     MSVCRT:gs_cookie.obj
 0003:00000028       __security_cookie_complement 0000000180009028     MSVCRT:gs_cookie.obj
 0003:00000030       __scrt_native_dllmain_reason 0000000180009030     MSVCRT:utility.obj
 0003:00000038       __isa_available            0000000180009038     MSVCRT:cpu_disp.obj
 0003:0000003c       __isa_enabled              000000018000903c     MSVCRT:cpu_disp.obj
 0003:00000040       __memset_fast_string_threshold 0000000180009040     MSVCRT:cpu_disp.obj
 0003:00000048       __memset_nt_threshold      0000000180009048     MSVCRT:cpu_disp.obj
 0003:00000050       __scrt_ucrt_dll_is_in_use  0000000180009050     MSVCRT:ucrt_stubs.obj
 0003:00000060       MethodNameStruct           0000000180009060     libIndyRedefineClass.obj
 0003:00000390       ?_OptionsStorage@?1??__local_stdio_printf_options@@9@4_KA 0000000180009390     libIndyRedefineClass.obj
 0003:00000958       _tls_index                 0000000180009958     MSVCRT:tlssup.obj
 0003:00000960       __scrt_current_native_startup_state 0000000180009960     MSVCRT:utility.obj
 0003:00000968       __scrt_native_startup_lock 0000000180009968     MSVCRT:utility.obj
 0003:000009a8       __scrt_debugger_hook_flag  00000001800099a8     MSVCRT:utility_desktop.obj
 0003:000009b0       ?__type_info_root_node@@3U__type_info_node@@A 00000001800099b0     MSVCRT:tncleanup.obj
 0003:000009c0       ?_OptionsStorage@?1??__local_stdio_scanf_options@@9@4_KA 00000001800099c0     MSVCRT:default_local_stdio_options.obj
 0003:000009c8       __favor                    00000001800099c8     MSVCRT:cpu_disp.obj
 0003:000009d0       __dyn_tls_init_callback    00000001800099d0     <common>

 entry point at        0001:000031e0

 Static symbols

 0000:ffff4000       .debug$S                   0000000180000000     IndyRedefineClass.exp
 0000:ffff4000       .debug$S                   0000000180000000     vcruntime:VCRUNTIME140.dll
 0000:ffff4000       .debug$S                   0000000180000000     vcruntime:VCRUNTIME140.dll
 0000:ffff4000       .debug$S                   0000000180000000     vcruntime:VCRUNTIME140.dll
 0000:ffff4000       .debug$S                   0000000180000000     vcruntime:VCRUNTIME140.dll
 0000:ffff4000       .debug$S                   0000000180000000     vcruntime:VCRUNTIME140.dll
 0000:ffff4000       .debug$S                   0000000180000000     vcruntime:VCRUNTIME140.dll
 0000:ffff4000       .debug$S                   0000000180000000     vcruntime:VCRUNTIME140.dll
 0000:ffff4000       .debug$S                   0000000180000000     ucrt:api-ms-win-crt-convert-l1-1-0.dll
 0000:ffff4000       .debug$S                   0000000180000000     ucrt:api-ms-win-crt-heap-l1-1-0.dll
 0000:ffff4000       .debug$S                   0000000180000000     ucrt:api-ms-win-crt-heap-l1-1-0.dll
 0000:ffff4000       .debug$S                   0000000180000000     ucrt:api-ms-win-crt-heap-l1-1-0.dll
 0000:ffff4000       .debug$S                   0000000180000000     ucrt:api-ms-win-crt-runtime-l1-1-0.dll
 0000:ffff4000       .debug$S                   0000000180000000     ucrt:api-ms-win-crt-runtime-l1-1-0.dll
 0000:ffff4000       .debug$S                   0000000180000000     ucrt:api-ms-win-crt-runtime-l1-1-0.dll
 0000:ffff4000       .debug$S                   0000000180000000     ucrt:api-ms-win-crt-runtime-l1-1-0.dll
 0000:ffff4000       .debug$S                   0000000180000000     ucrt:api-ms-win-crt-runtime-l1-1-0.dll
 0000:ffff4000       .debug$S                   0000000180000000     ucrt:api-ms-win-crt-runtime-l1-1-0.dll
 0000:ffff4000       .debug$S                   0000000180000000     ucrt:api-ms-win-crt-runtime-l1-1-0.dll
 0000:ffff4000       .debug$S                   0000000180000000     ucrt:api-ms-win-crt-runtime-l1-1-0.dll
 0000:ffff4000       .debug$S                   0000000180000000     ucrt:api-ms-win-crt-runtime-l1-1-0.dll
 0000:ffff4000       .debug$S                   0000000180000000     ucrt:api-ms-win-crt-runtime-l1-1-0.dll
 0000:ffff4000       .debug$S                   0000000180000000     ucrt:api-ms-win-crt-runtime-l1-1-0.dll
 0000:ffff4000       .debug$S                   0000000180000000     ucrt:api-ms-win-crt-runtime-l1-1-0.dll
 0000:ffff4000       .debug$S                   0000000180000000     ucrt:api-ms-win-crt-runtime-l1-1-0.dll
 0000:ffff4000       .debug$S                   0000000180000000     ucrt:api-ms-win-crt-runtime-l1-1-0.dll
 0000:ffff4000       .debug$S                   0000000180000000     ucrt:api-ms-win-crt-runtime-l1-1-0.dll
 0000:ffff4000       .debug$S                   0000000180000000     ucrt:api-ms-win-crt-runtime-l1-1-0.dll
 0000:ffff4000       .debug$S                   0000000180000000     ucrt:api-ms-win-crt-stdio-l1-1-0.dll
 0000:ffff4000       .debug$S                   0000000180000000     ucrt:api-ms-win-crt-stdio-l1-1-0.dll
 0000:ffff4000       .debug$S                   0000000180000000     ucrt:api-ms-win-crt-stdio-l1-1-0.dll
 0000:ffff4000       .debug$S                   0000000180000000     ucrt:api-ms-win-crt-stdio-l1-1-0.dll
 0000:ffff4000       .debug$S                   0000000180000000     ucrt:api-ms-win-crt-stdio-l1-1-0.dll
 0000:ffff4000       .debug$S                   0000000180000000     ucrt:api-ms-win-crt-stdio-l1-1-0.dll
 0000:ffff4000       .debug$S                   0000000180000000     ucrt:api-ms-win-crt-stdio-l1-1-0.dll
 0000:ffff4000       .debug$S                   0000000180000000     ucrt:api-ms-win-crt-stdio-l1-1-0.dll
 0000:ffff4000       .debug$S                   0000000180000000     ucrt:api-ms-win-crt-stdio-l1-1-0.dll
 0000:ffff4000       .debug$S                   0000000180000000     ucrt:api-ms-win-crt-stdio-l1-1-0.dll
 0000:ffff4000       .debug$S                   0000000180000000     ucrt:api-ms-win-crt-string-l1-1-0.dll
 0000:ffff4000       .debug$S                   0000000180000000     ucrt:api-ms-win-crt-string-l1-1-0.dll
 0000:ffff4000       .debug$S                   0000000180000000     ucrt:api-ms-win-crt-string-l1-1-0.dll
 0000:ffff4000       .debug$S                   0000000180000000     ucrt:api-ms-win-crt-string-l1-1-0.dll
 0000:ffff4000       .debug$S                   0000000180000000     ucrt:api-ms-win-crt-string-l1-1-0.dll
 0000:ffff4000       .debug$S                   0000000180000000     ucrt:api-ms-win-crt-string-l1-1-0.dll
 0000:ffff4000       .debug$S                   0000000180000000     ucrt:api-ms-win-crt-string-l1-1-0.dll
 0000:ffff4000       .debug$S                   0000000180000000     ucrt:api-ms-win-crt-string-l1-1-0.dll
 0000:ffff4000       .debug$S                   0000000180000000     kernel32:KERNEL32.dll
 0000:ffff4000       .debug$S                   0000000180000000     kernel32:KERNEL32.dll
 0000:ffff4000       .debug$S                   0000000180000000     kernel32:KERNEL32.dll
 0000:ffff4000       .debug$S                   0000000180000000     kernel32:KERNEL32.dll
 0000:ffff4000       .debug$S                   0000000180000000     kernel32:KERNEL32.dll
 0000:ffff4000       .debug$S                   0000000180000000     kernel32:KERNEL32.dll
 0000:ffff4000       .debug$S                   0000000180000000     kernel32:KERNEL32.dll
 0000:ffff4000       .debug$S                   0000000180000000     kernel32:KERNEL32.dll
 0000:ffff4000       .debug$S                   0000000180000000     kernel32:KERNEL32.dll
 0000:ffff4000       .debug$S                   0000000180000000     kernel32:KERNEL32.dll
 0000:ffff4000       .debug$S                   0000000180000000     kernel32:KERNEL32.dll
 0000:ffff4000       .debug$S                   0000000180000000     kernel32:KERNEL32.dll
 0000:ffff4000       .debug$S                   0000000180000000     kernel32:KERNEL32.dll
 0000:ffff4000       .debug$S                   0000000180000000     kernel32:KERNEL32.dll
 0000:ffff4000       .debug$S                   0000000180000000     kernel32:KERNEL32.dll
 0000:ffff4000       .debug$S                   0000000180000000     kernel32:KERNEL32.dll
 0000:ffff4000       .debug$S                   0000000180000000     kernel32:KERNEL32.dll
 0000:ffff4000       .debug$S                   0000000180000000     kernel32:KERNEL32.dll
 0000:ffff4000       .debug$S                   0000000180000000     kernel32:KERNEL32.dll
 0000:ffff4000       .debug$S                   0000000180000000     kernel32:KERNEL32.dll
 0000:ffff4000       .debug$S                   0000000180000000     kernel32:KERNEL32.dll
 0000:ffff4000       .debug$S                   0000000180000000     kernel32:KERNEL32.dll
 0000:ffff4000       .debug$S                   0000000180000000     kernel32:KERNEL32.dll
 0000:ffff4000       .debug$S                   0000000180000000     kernel32:KERNEL32.dll
 0000:ffff4000       .debug$S                   0000000180000000     kernel32:KERNEL32.dll
 0000:ffff4000       .debug$S                   0000000180000000     kernel32:KERNEL32.dll
 0000:ffff4000       .debug$S                   0000000180000000     kernel32:KERNEL32.dll
 0000:ffff4000       .debug$S                   0000000180000000     kernel32:KERNEL32.dll
 0001:00000bfc       MethodEntry                0000000180001bfc f   libIndyRedefineClass.obj
 0001:00000ddc       SingleStep                 0000000180001ddc f   libIndyRedefineClass.obj
 0001:00000ec8       agentThreadWrapper         0000000180001ec8 f   libIndyRedefineClass.obj
 0001:00001034       check_option               0000000180002034 f   libIndyRedefineClass.obj
 0001:00001364       file_basename              0000000180002364 f   libIndyRedefineClass.obj
 0001:00002418       popFrameLogic              0000000180003418 f   libIndyRedefineClass.obj
 0001:000026bc       startAgentThreadWrapper    00000001800036bc f   libIndyRedefineClass.obj
 0001:000029fc       syncDebuggeeStatus         00000001800039fc f   libIndyRedefineClass.obj
 0001:00002c9c       capture_previous_context   0000000180003c9c f   MSVCRT:gs_report.obj
 0001:00002d10       ?__scrt_initialize_thread_safe_statics@@YAHXZ 0000000180003d10 f   MSVCRT:thread_safe_statics.obj
 0001:00002de0       ?__scrt_uninitialize_thread_safe_statics@@YAXXZ 0000000180003de0 f   MSVCRT:thread_safe_statics.obj
 0001:00002e90       $$000000                   0000000180003e90     MSVCRT:amdsecgs.obj
 0001:00002ec0       ?dllmain_crt_dispatch@@YAHQEAUHINSTANCE__@@KQEAX@Z 0000000180003ec0 f   MSVCRT:dll_dllmain.obj
 0001:00002f10       ?dllmain_crt_process_attach@@YAHQEAUHINSTANCE__@@QEAX@Z 0000000180003f10 f   MSVCRT:dll_dllmain.obj
 0001:00003028       ?dllmain_crt_process_detach@@YAH_N@Z 0000000180004028 f   MSVCRT:dll_dllmain.obj
 0001:000030ac       ?dllmain_dispatch@@YAHQEAUHINSTANCE__@@KQEAX@Z 00000001800040ac f   MSVCRT:dll_dllmain.obj
 0001:00003ac0       $$000000                   0000000180004ac0     MSVCRT:guard_dispatch.obj
 0001:00003ae0       $$000000                   0000000180004ae0     MSVCRT:guard_xfg_dispatch.obj
 0001:00003af6       ?fin$0@?0??dllmain_crt_process_attach@@YAHQEAUHINSTANCE__@@QEAX@Z@4HA 0000000180004af6 f   MSVCRT:dll_dllmain.obj
 0001:00003b0d       ?fin$0@?0??dllmain_crt_process_detach@@YAH_N@Z@4HA 0000000180004b0d f   MSVCRT:dll_dllmain.obj
 0001:00003b26       ?fin$1@?0??dllmain_crt_process_detach@@YAH_N@Z@4HA 0000000180004b26 f   MSVCRT:dll_dllmain.obj
 0001:00003b3a       ?filt$0@?0??dllmain_dispatch@@YAHQEAUHINSTANCE__@@KQEAX@Z@4HA 0000000180004b3a f   MSVCRT:dll_dllmain.obj
 0001:00003b70       __scrt_is_nonwritable_in_current_image$filt$0 0000000180004b70 f   MSVCRT:utility.obj
 0002:00000248       ?__scrt_initialize_tss_var@@3P6AHXZEA 0000000180005248     MSVCRT:thread_safe_statics.obj
 0002:00001e28       GS_ExceptionPointers       0000000180006e28     MSVCRT:gs_report.obj
 0002:00002528       $unwind$fprintf            0000000180007528     libIndyRedefineClass.obj
 0002:00002534       $unwind$printf             0000000180007534     libIndyRedefineClass.obj
 0002:00002540       $unwind$_snprintf          0000000180007540     libIndyRedefineClass.obj
 0002:00002550       $unwind$?NewObject@JNIEnv_@@QEAAPEAV_jobject@@PEAV_jclass@@PEAU_jmethodID@@ZZ 0000000180007550     libIndyRedefineClass.obj
 0002:00002550       $unwind$nsk_lcomplain      0000000180007550     libIndyRedefineClass.obj
 0002:00002550       $unwind$nsk_ldisplay       0000000180007550     libIndyRedefineClass.obj
 0002:00002558       $unwind$nsk_lvdisplay      0000000180007558     libIndyRedefineClass.obj
 0002:00002558       $unwind$_RTC_Initialize    0000000180007558     MSVCRT:initsect.obj
 0002:00002558       $unwind$_RTC_Terminate     0000000180007558     MSVCRT:initsect.obj
 0002:00002558       $unwind$?__scrt_initialize_thread_safe_statics@@YAHXZ 0000000180007558     MSVCRT:thread_safe_statics.obj
 0002:00002564       $unwind$nsk_complain       0000000180007564     libIndyRedefineClass.obj
 0002:00002564       $unwind$nsk_printf         0000000180007564     libIndyRedefineClass.obj
 0002:0000256c       $unwind$nsk_lvcomplain     000000018000756c     libIndyRedefineClass.obj
 0002:00002584       $unwind$nsk_ltrace         0000000180007584     libIndyRedefineClass.obj
 0002:00002584       $unwind$__report_gsfailure 0000000180007584     MSVCRT:gs_report.obj
 0002:0000258c       $unwind$Java_vm_mlvm_indy_func_jvmti_share_IndyRedefineClass_checkStatus 000000018000758c     libIndyRedefineClass.obj
 0002:0000258c       $unwind$nsk_lvtrace        000000018000758c     libIndyRedefineClass.obj
 0002:0000258c       $unwind$__raise_securityfailure 000000018000758c     MSVCRT:gs_report.obj
 0002:0000258c       $unwind$__scrt_initialize_crt 000000018000758c     MSVCRT:utility.obj
 0002:0000258c       $unwind$__scrt_initialize_onexit_tables 000000018000758c     MSVCRT:utility.obj
 0002:0000258c       $unwind$__scrt_release_startup_lock 000000018000758c     MSVCRT:utility.obj
 0002:0000258c       $unwind$__scrt_uninitialize_crt 000000018000758c     MSVCRT:utility.obj
 0002:0000258c       $unwind$_onexit            000000018000758c     MSVCRT:utility.obj
 0002:00002594       $unwind$nsk_lverify        0000000180007594     libIndyRedefineClass.obj
 0002:000025a4       $unwind$nsk_vprintf        00000001800075a4     libIndyRedefineClass.obj
 0002:000025b4       $unwind$?nsk_jni_lverify@@YAHHPEAUJNIEnv_@@HQEBDH1ZZ 00000001800075b4     libIndyRedefineClass.obj
 0002:000025c8       $unwind$?nsk_jni_check_exception@@YAHPEAUJNIEnv_@@QEBDH@Z 00000001800075c8     libIndyRedefineClass.obj
 0002:000025e4       $unwind$nsk_jvmti_parseOptions 00000001800075e4     libIndyRedefineClass.obj
 0002:00002600       $unwind$nsk_jvmti_createJVMTIEnv 0000000180007600     libIndyRedefineClass.obj
 0002:00002614       $unwind$Java_vm_mlvm_indy_func_jvmti_share_IndyRedefineClass_setRedefineTriggerMethodName 0000000180007614     libIndyRedefineClass.obj
 0002:00002614       $unwind$Java_vm_mlvm_indy_func_jvmti_share_IndyRedefineClass_setRedefinedClassFileName 0000000180007614     libIndyRedefineClass.obj
 0002:00002614       $unwind$nsk_jvmti_resetAgentData 0000000180007614     libIndyRedefineClass.obj
 0002:00002614       $unwind$nsk_jvmti_setFailStatus 0000000180007614     libIndyRedefineClass.obj
 0002:00002614       $unwind$__scrt_initialize_default_local_stdio_options 0000000180007614     MSVCRT:default_local_stdio_options.obj
 0002:00002614       $unwind$?dllmain_crt_dispatch@@YAHQEAUHINSTANCE__@@KQEAX@Z 0000000180007614     MSVCRT:dll_dllmain.obj
 0002:00002614       $unwind$DllMain            0000000180007614     MSVCRT:dll_dllmain_stub.obj
 0002:00002614       $unwind$__GSHandlerCheck   0000000180007614     MSVCRT:gshandler.obj
 0002:00002614       $unwind$?__scrt_uninitialize_thread_safe_statics@@YAXXZ 0000000180007614     MSVCRT:thread_safe_statics.obj
 0002:00002614       $unwind$__scrt_acquire_startup_lock 0000000180007614     MSVCRT:utility.obj
 0002:00002614       $unwind$__scrt_dllmain_after_initialize_c 0000000180007614     MSVCRT:utility.obj
 0002:00002614       $unwind$__scrt_dllmain_before_initialize_c 0000000180007614     MSVCRT:utility.obj
 0002:00002614       $unwind$__scrt_dllmain_crt_thread_attach 0000000180007614     MSVCRT:utility.obj
 0002:00002614       $unwind$__scrt_dllmain_crt_thread_detach 0000000180007614     MSVCRT:utility.obj
 0002:00002614       $unwind$__scrt_dllmain_uninitialize_c 0000000180007614     MSVCRT:utility.obj
 0002:00002614       $unwind$__scrt_dllmain_uninitialize_critical 0000000180007614     MSVCRT:utility.obj
 0002:00002614       $unwind$atexit             0000000180007614     MSVCRT:utility.obj
 0002:0000261c       $unwind$SingleStep         000000018000761c     libIndyRedefineClass.obj
 0002:0000261c       $unwind$check_option       000000018000761c     libIndyRedefineClass.obj
 0002:0000261c       $unwind$nsk_jvmti_findOptionValue 000000018000761c     libIndyRedefineClass.obj
 0002:0000261c       $unwind$_DllMainCRTStartup 000000018000761c     MSVCRT:dll_dllmain.obj
 0002:0000262c       $unwind$nsk_jvmti_lverify  000000018000762c     libIndyRedefineClass.obj
 0002:00002640       $unwind$nsk_jvmti_redefineClass 0000000180007640     libIndyRedefineClass.obj
 0002:00002660       $unwind$??1JvmtiResource@@QEAA@XZ 0000000180007660     libIndyRedefineClass.obj
 0002:00002660       $unwind$exitOnError        0000000180007660     libIndyRedefineClass.obj
 0002:00002670       $unwind$Agent_Initialize   0000000180007670     libIndyRedefineClass.obj
 0002:00002694       $unwind$Java_nsk_share_jvmti_DebugeeClass_checkStatus 0000000180007694     libIndyRedefineClass.obj
 0002:00002694       $unwind$agentThreadWrapper 0000000180007694     libIndyRedefineClass.obj
 0002:000026a4       $unwind$startAgentThreadWrapper 00000001800076a4     libIndyRedefineClass.obj
 0002:000026c0       $unwind$syncDebuggeeStatus 00000001800076c0     libIndyRedefineClass.obj
 0002:000026c0       $unwind$__scrt_dllmain_exception_filter 00000001800076c0     MSVCRT:utility.obj
 0002:000026d4       $unwind$Java_nsk_share_jvmti_DebugeeClass_resetAgentData 00000001800076d4     libIndyRedefineClass.obj
 0002:000026dc       $unwind$MA_checkStatus     00000001800076dc     libIndyRedefineClass.obj
 0002:000026f0       $unwind$Java_nsk_share_jvmti_ArgumentHandler_getAgentOptionsString 00000001800076f0     libIndyRedefineClass.obj
 0002:00002704       $unwind$copyFromJString    0000000180007704     libIndyRedefineClass.obj
 0002:0000271c       $unwind$getMethodName      000000018000771c     libIndyRedefineClass.obj
 0002:00002730       $unwind$locationToString   0000000180007730     libIndyRedefineClass.obj
 0002:00002748       $unwind$getTLS             0000000180007748     libIndyRedefineClass.obj
 0002:00002764       $unwind$popFrameLogic      0000000180007764     libIndyRedefineClass.obj
 0002:00002780       $unwind$MethodEntry        0000000180007780     libIndyRedefineClass.obj
 0002:0000279c       $unwind$capture_previous_context 000000018000779c     MSVCRT:gs_report.obj
 0002:000027a8       $unwind$__GSHandlerCheckCommon 00000001800077a8     MSVCRT:gshandler.obj
 0002:000027b0       $xdatasym                  00000001800077b0     MSVCRT:amdsecgs.obj
 0002:000027b4       $unwind$?dllmain_crt_process_attach@@YAHQEAUHINSTANCE__@@QEAX@Z 00000001800077b4     MSVCRT:dll_dllmain.obj
 0002:000027f0       $unwind$?fin$0@?0??dllmain_crt_process_attach@@YAHQEAUHINSTANCE__@@QEAX@Z@4HA 00000001800077f0     MSVCRT:dll_dllmain.obj
 0002:000027f0       $unwind$?fin$0@?0??dllmain_crt_process_detach@@YAH_N@Z@4HA 00000001800077f0     MSVCRT:dll_dllmain.obj
 0002:000027f0       $unwind$?fin$1@?0??dllmain_crt_process_detach@@YAH_N@Z@4HA 00000001800077f0     MSVCRT:dll_dllmain.obj
 0002:000027f8       $unwind$?dllmain_crt_process_detach@@YAH_N@Z 00000001800077f8     MSVCRT:dll_dllmain.obj
 0002:0000284c       $unwind$?dllmain_dispatch@@YAHQEAUHINSTANCE__@@KQEAX@Z 000000018000784c     MSVCRT:dll_dllmain.obj
 0002:00002874       $unwind$?filt$0@?0??dllmain_dispatch@@YAHQEAUHINSTANCE__@@KQEAX@Z@4HA 0000000180007874     MSVCRT:dll_dllmain.obj
 0002:0000287c       $unwind$__scrt_is_nonwritable_in_current_image 000000018000787c     MSVCRT:utility.obj
 0002:0000289c       $unwind$__scrt_is_nonwritable_in_current_image$filt$0 000000018000789c     MSVCRT:utility.obj
 0002:000028a4       $unwind$__scrt_fastfail    00000001800078a4     MSVCRT:utility_desktop.obj
 0002:000028b4       $unwind$__security_init_cookie 00000001800078b4     MSVCRT:gs_support.obj
 0002:000028c0       $unwind$__isa_available_init 00000001800078c0     MSVCRT:cpu_disp.obj
 0002:000028d0       $xdatasym                  00000001800078d0     MSVCRT:guard_dispatch.obj
 0002:000028d8       $xdatasym                  00000001800078d8     MSVCRT:guard_xfg_dispatch.obj
 0002:000028e0       .edata                     00000001800078e0     IndyRedefineClass.exp
 0002:00002908       rgpv                       0000000180007908     IndyRedefineClass.exp
 0002:0000293c       rgszName                   000000018000793c     IndyRedefineClass.exp
 0002:00002970       rgwOrd                     0000000180007970     IndyRedefineClass.exp
 0002:0000298a       szName                     000000018000798a     IndyRedefineClass.exp
 0002:000029a0       $N00001                    00000001800079a0     IndyRedefineClass.exp
 0002:000029af       $N00002                    00000001800079af     IndyRedefineClass.exp
 0002:000029bc       $N00003                    00000001800079bc     IndyRedefineClass.exp
 0002:000029f7       $N00004                    00000001800079f7     IndyRedefineClass.exp
 0002:00002a25       $N00005                    0000000180007a25     IndyRedefineClass.exp
 0002:00002a56       $N00006                    0000000180007a56     IndyRedefineClass.exp
 0002:00002a85       $N00007                    0000000180007a85     IndyRedefineClass.exp
 0002:00002ab4       $N00008                    0000000180007ab4     IndyRedefineClass.exp
 0002:00002ae9       $N00009                    0000000180007ae9     IndyRedefineClass.exp
 0002:00002b2a       $N00010                    0000000180007b2a     IndyRedefineClass.exp
 0002:00002b7d       $N00011                    0000000180007b7d     IndyRedefineClass.exp
 0002:00002bcf       $N00012                    0000000180007bcf     IndyRedefineClass.exp
 0002:00002c1e       $N00013                    0000000180007c1e     IndyRedefineClass.exp
 0002:000030b2       .idata$6                   00000001800080b2     kernel32:KERNEL32.dll
 0002:0000310c       .idata$6                   000000018000810c     vcruntime:VCRUNTIME140.dll
 0002:000032d2       .idata$6                   00000001800082d2     ucrt:api-ms-win-crt-stdio-l1-1-0.dll
 0002:000032f2       .idata$6                   00000001800082f2     ucrt:api-ms-win-crt-runtime-l1-1-0.dll
 0002:00003314       .idata$6                   0000000180008314     ucrt:api-ms-win-crt-heap-l1-1-0.dll
 0002:00003334       .idata$6                   0000000180008334     ucrt:api-ms-win-crt-convert-l1-1-0.dll
 0002:00003356       .idata$6                   0000000180008356     ucrt:api-ms-win-crt-string-l1-1-0.dll
 0003:00000000       gPopFrameDepth             0000000180009000     libIndyRedefineClass.obj
 0003:00000008       gszRedefineTriggerMethodName 0000000180009008     libIndyRedefineClass.obj
 0003:00000010       gszRedefinedClassFileName  0000000180009010     libIndyRedefineClass.obj
 0003:00000260       nsk_context                0000000180009260     libIndyRedefineClass.obj
 0003:0000026c       currentAgentStatus         000000018000926c     libIndyRedefineClass.obj
 0003:00000270       agentThread                0000000180009270     libIndyRedefineClass.obj
 0003:00000278       agentThreadProc            0000000180009278     libIndyRedefineClass.obj
 0003:00000280       agentThreadArg             0000000180009280     libIndyRedefineClass.obj
 0003:00000288       agent_data                 0000000180009288     libIndyRedefineClass.obj
 0003:00000298       jvmti_env                  0000000180009298     libIndyRedefineClass.obj
 0003:000002a0       jvm                        00000001800092a0     libIndyRedefineClass.obj
 0003:000002a8       jni_env                    00000001800092a8     libIndyRedefineClass.obj
 0003:000002b0       checkStatus_func           00000001800092b0     libIndyRedefineClass.obj
 0003:000002b8       redefineAttempted          00000001800092b8     libIndyRedefineClass.obj
 0003:000002bc       redefineSucceed            00000001800092bc     libIndyRedefineClass.obj
 0003:000002c0       agentFailed                00000001800092c0     libIndyRedefineClass.obj
 0003:000002c4       gIsMethodEntryWorking      00000001800092c4     libIndyRedefineClass.obj
 0003:000002c5       gIsSingleStepWorking       00000001800092c5     libIndyRedefineClass.obj
 0003:000002c6       gIsErrorOccured            00000001800092c6     libIndyRedefineClass.obj
 0003:000002c7       gIsDebuggerCompatible      00000001800092c7     libIndyRedefineClass.obj
 0003:000002c8       gJvmtiEnv                  00000001800092c8     libIndyRedefineClass.obj
 0003:000002d0       context                    00000001800092d0     libIndyRedefineClass.obj
 0003:00000388       gIsClassRedefined          0000000180009388     libIndyRedefineClass.obj
 0003:000003a0       GS_ExceptionRecord         00000001800093a0     MSVCRT:gs_report.obj
 0003:00000440       GS_ContextRecord           0000000180009440     MSVCRT:gs_report.obj
 0003:00000910       ?g_tss_cv@@3U_RTL_CONDITION_VARIABLE@@A 0000000180009910     MSVCRT:thread_safe_statics.obj
 0003:00000918       ?g_tss_event@@3PEAXEA      0000000180009918     MSVCRT:thread_safe_statics.obj
 0003:00000920       ?g_tss_mutex@@3U_RTL_CRITICAL_SECTION@@A 0000000180009920     MSVCRT:thread_safe_statics.obj
 0003:00000948       ?g_sleep_condition_variable_cs@@3P6AHPEAU_RTL_CONDITION_VARIABLE@@PEAU_RTL_CRITICAL_SECTION@@K@ZEA 0000000180009948     MSVCRT:thread_safe_statics.obj
 0003:00000950       ?g_wake_all_condition_variable@@3P6AXPEAU_RTL_CONDITION_VARIABLE@@@ZEA 0000000180009950     MSVCRT:thread_safe_statics.obj
 0003:0000095c       ?__proc_attached@@3HA      000000018000995c     MSVCRT:dll_dllmain.obj
 0003:00000970       ?is_initialized_as_dll@@3_NA 0000000180009970     MSVCRT:utility.obj
 0003:00000971       ?module_local_atexit_table_initialized@@3_NA 0000000180009971     MSVCRT:utility.obj
 0003:00000978       ?module_local_atexit_table@@3U_onexit_table_t@@A 0000000180009978     MSVCRT:utility.obj
 0003:00000990       ?module_local_at_quick_exit_table@@3U_onexit_table_t@@A 0000000180009990     MSVCRT:utility.obj
